BL51 BANKED LINKER/LOCATER V5.03                                                        07/06/2006  17:26:57  PAGE 1


BL51 BANKED LINKER/LOCATER V5.03, INVOKED BY:
C:\KEIL\C51\BIN\BL51.EXE STARTUP.obj, gLCD_STK1_Demo1.obj, delay.obj, ks0108.obj TO JHD12864_demo1 RAMSIZE (256) CODE (0
>> X0000-0X1FFF)


MEMORY MODEL: SMALL


INPUT MODULES INCLUDED:
  STARTUP.obj (?C_STARTUP)
  gLCD_STK1_Demo1.obj (GLCD_STK1_DEMO1)
  delay.obj (DELAY)
  ks0108.obj (KS0108)
  C:\KEIL\C51\LIB\C51S.LIB (?C?CLDPTR)


LINK MAP OF MODULE:  JHD12864_demo1 (?C_STARTUP)


            TYPE    BASE      LENGTH    RELOCATION   SEGMENT NAME
            -----------------------------------------------------

            * * * * * * *   D A T A   M E M O R Y   * * * * * * *
            REG     0000H     0008H     ABSOLUTE     "REG BANK 0"
            DATA    0008H     0011H     UNIT         _DATA_GROUP_
                    0019H     0007H                  *** GAP ***
            BIT     0020H.0   0000H.3   UNIT         _BIT_GROUP_
                    0020H.3   0000H.5                *** GAP ***
            IDATA   0021H     0001H     UNIT         ?STACK

            * * * * * * *   C O D E   M E M O R Y   * * * * * * *
            CODE    0000H     0003H     ABSOLUTE     
                    0003H     07FDH                  *** GAP ***
            CODE    0800H     0357H     UNIT         ?CO?KS0108
            CODE    0B57H     00DFH     UNIT         ?PR?MAIN?GLCD_STK1_DEMO1
            CODE    0C36H     00DDH     UNIT         ?PR?_GDISPPIXSTRAT?KS0108
            CODE    0D13H     0091H     UNIT         ?CO?GLCD_STK1_DEMO1
            CODE    0DA4H     007FH     UNIT         ?PR?_GDISPSETPIXEL?KS0108
            CODE    0E23H     0044H     UNIT         ?PR?_GDISPWRBYTE?KS0108
            CODE    0E67H     0024H     UNIT         ?PR?_GDISPCLR?KS0108
            CODE    0E8BH     0020H     UNIT         ?PR?_DELAYMS?DELAY
            CODE    0EABH     0020H     UNIT         ?PR?_GDISPCHIPSEL?KS0108
            CODE    0ECBH     001FH     UNIT         ?PR?GDISPINIT?KS0108
            CODE    0EEAH     001CH     UNIT         ?PR?GDISPSWITCH?KS0108
            CODE    0F06H     001CH     UNIT         ?PR?GDISPWR?KS0108
            CODE    0F22H     0019H     UNIT         ?C?LIB_CODE
            CODE    0F3BH     0016H     UNIT         ?PR?GDISPRD?KS0108
            CODE    0F51H     0012H     UNIT         ?PR?_DELAYUS?DELAY
            CODE    0F63H     0011H     UNIT         ?PR?GDISPRESET?KS0108
            CODE    0F74H     000CH     UNIT         ?C_C51STARTUP
            CODE    0F80H     0009H     UNIT         ?PR?GDISPBACKLITE?KS0108



OVERLAY MAP OF MODULE:   JHD12864_demo1 (?C_STARTUP)


SEGMENT                              BIT_GROUP          DATA_GROUP 
BL51 BANKED LINKER/LOCATER V5.03                                                      07/06/2006  17:26:57  PAGE 2


  +--> CALLED SEGMENT             START    LENGTH     START    LENGTH
---------------------------------------------------------------------
?C_C51STARTUP                     -----    -----      -----    -----
  +--> ?PR?MAIN?GLCD_STK1_DEMO1

?PR?MAIN?GLCD_STK1_DEMO1          -----    -----      0008H    0001H
  +--> ?PR?GDISPINIT?KS0108
  +--> ?CO?GLCD_STK1_DEMO1
  +--> ?PR?_GDISPPIXSTRAT?KS0108
  +--> ?PR?_GDISPSETPIXEL?KS0108
  +--> ?PR?_DELAYMS?DELAY
  +--> ?PR?_GDISPCLR?KS0108

?PR?GDISPINIT?KS0108              -----    -----      -----    -----
  +--> ?PR?GDISPBACKLITE?KS0108
  +--> ?PR?GDISPRESET?KS0108
  +--> ?PR?GDISPSWITCH?KS0108
  +--> ?PR?GDISPWR?KS0108
  +--> ?PR?_GDISPCLR?KS0108

?PR?GDISPBACKLITE?KS0108          0020H.0  0000H.1    -----    -----

?PR?GDISPSWITCH?KS0108            0020H.0  0000H.1    -----    -----
  +--> ?PR?_GDISPCHIPSEL?KS0108
  +--> ?PR?GDISPWR?KS0108

?PR?GDISPWR?KS0108                0020H.2  0000H.1    0018H    0001H

?PR?_GDISPCLR?KS0108              -----    -----      0009H    0003H
  +--> ?PR?_GDISPWRBYTE?KS0108

?PR?_GDISPWRBYTE?KS0108           -----    -----      000CH    0003H
  +--> ?PR?_GDISPCHIPSEL?KS0108
  +--> ?PR?GDISPWR?KS0108

?PR?_GDISPPIXSTRAT?KS0108         0020H.0  0000H.1    0009H    000CH
  +--> ?CO?KS0108
  +--> ?PR?_GDISPSETPIXEL?KS0108

?PR?_GDISPSETPIXEL?KS0108         0020H.1  0000H.1    0015H    0003H
  +--> ?PR?_GDISPCHIPSEL?KS0108
  +--> ?PR?GDISPWR?KS0108
  +--> ?PR?GDISPRD?KS0108

?PR?GDISPRD?KS0108                0020H.2  0000H.1    -----    -----



SYMBOL TABLE OF MODULE:  JHD12864_demo1 (?C_STARTUP)

  VALUE           TYPE          NAME
  ----------------------------------

  -------         MODULE        ?C_STARTUP
  C:0F74H         SEGMENT       ?C_C51STARTUP
  I:0021H         SEGMENT       ?STACK
  C:0000H         PUBLIC        ?C_STARTUP
BL51 BANKED LINKER/LOCATER V5.03                                                      07/06/2006  17:26:57  PAGE 3


  D:00E0H         SYMBOL        ACC
  D:00F0H         SYMBOL        B
  D:0083H         SYMBOL        DPH
  D:0082H         SYMBOL        DPL
  N:0000H         SYMBOL        IBPSTACK
  N:0100H         SYMBOL        IBPSTACKTOP
  N:0080H         SYMBOL        IDATALEN
  C:0F77H         SYMBOL        IDATALOOP
  N:0000H         SYMBOL        PBPSTACK
  N:0000H         SYMBOL        PBPSTACKTOP
  N:0000H         SYMBOL        PDATALEN
  N:0000H         SYMBOL        PDATASTART
  N:0000H         SYMBOL        PPAGE
  N:0000H         SYMBOL        PPAGEENABLE
  D:00A0H         SYMBOL        PPAGE_SFR
  D:0081H         SYMBOL        SP
  C:0F74H         SYMBOL        STARTUP1
  N:0000H         SYMBOL        XBPSTACK
  N:0000H         SYMBOL        XBPSTACKTOP
  N:0000H         SYMBOL        XDATALEN
  N:0000H         SYMBOL        XDATASTART
  C:0000H         LINE#         92
  C:0F74H         LINE#         99
  C:0F76H         LINE#         100
  C:0F77H         LINE#         101
  C:0F78H         LINE#         102
  C:0F7AH         LINE#         151
  C:0F7DH         LINE#         155
  -------         ENDMOD        ?C_STARTUP

  -------         MODULE        GLCD_STK1_DEMO1
  C:0000H         SYMBOL        _ICE_DUMMY_
  D:00A0H         PUBLIC        P2
  C:0B57H         PUBLIC        main
  -------         PROC          MAIN
  -------         DO            
  D:0008H         SYMBOL        x
  -------         ENDDO         
  C:0B57H         LINE#         18
  C:0B57H         LINE#         19
  C:0B57H         LINE#         22
  C:0B5AH         LINE#         24
  C:0B5AH         LINE#         25
  C:0B6CH         LINE#         26
  C:0B7EH         LINE#         27
  C:0B93H         LINE#         28
  C:0BA8H         LINE#         29
  C:0BAFH         LINE#         30
  C:0BB4H         LINE#         31
  C:0BC6H         LINE#         32
  C:0BD8H         LINE#         33
  C:0BEDH         LINE#         34
  C:0C02H         LINE#         35
  C:0C09H         LINE#         36
  C:0C0EH         LINE#         37
  C:0C15H         LINE#         38
  C:0C27H         LINE#         39
BL51 BANKED LINKER/LOCATER V5.03                                                      07/06/2006  17:26:57  PAGE 4


  C:0C2EH         LINE#         40
  C:0C33H         LINE#         41
  -------         ENDPROC       MAIN
  -------         ENDMOD        GLCD_STK1_DEMO1

  -------         MODULE        DELAY
  C:0000H         SYMBOL        _ICE_DUMMY_
  D:0090H         PUBLIC        P1
  D:00B0H         PUBLIC        P3
  D:00A8H         PUBLIC        IE
  C:0E8BH         PUBLIC        _DelayMs
  D:00B8H         PUBLIC        IP
  C:0F51H         PUBLIC        _DelayUs
  D:0098H         PUBLIC        SCON
  D:0088H         PUBLIC        TCON
  D:00C8H         PUBLIC        T2CON
  D:00D0H         PUBLIC        PSW
  -------         PROC          _DELAYUS
  D:0006H         SYMBOL        N
  -------         DO            
  D:0004H         SYMBOL        x
  -------         ENDDO         
  C:0F51H         LINE#         36
  C:0F51H         LINE#         37
  C:0F51H         LINE#         40
  C:0F62H         LINE#         41
  -------         ENDPROC       _DELAYUS
  -------         PROC          _DELAYMS
  D:0006H         SYMBOL        msec
  -------         DO            
  D:0004H         SYMBOL        x
  D:0002H         SYMBOL        y
  -------         ENDDO         
  C:0E8BH         LINE#         54
  C:0E8BH         LINE#         55
  C:0E8BH         LINE#         58
  C:0E95H         LINE#         59
  C:0E95H         LINE#         60
  C:0EA3H         LINE#         61
  C:0EAAH         LINE#         62
  -------         ENDPROC       _DELAYMS
  -------         ENDMOD        DELAY

  -------         MODULE        KS0108
  C:0000H         SYMBOL        _ICE_DUMMY_
  D:0080H         PUBLIC        P0
  D:00A0H         PUBLIC        P2
  C:0F3BH         PUBLIC        GDispRd
  C:0E23H         PUBLIC        _GDispWrByte
  C:0F0EH         PUBLIC        GDispWr
  B:00A0H.6       PUBLIC        LCD_RST
  B:00A0H.1       PUBLIC        LCD_DI
  B:00A0H.7       PUBLIC        LCD_BL
  B:00A0H.3       PUBLIC        LCD_EN
  C:0800H         PUBLIC        SYS_FNT
  C:0EEAH         PUBLIC        GDispSwitch
  C:0E67H         PUBLIC        _GDispClr
BL51 BANKED LINKER/LOCATER V5.03                                                      07/06/2006  17:26:57  PAGE 5


  B:00A0H.2       PUBLIC        LCD_RW
  C:0F80H         PUBLIC        GDispBackLite
  C:0C36H         PUBLIC        _GDispPixStrAt
  C:0F63H         PUBLIC        GDispReset
  C:0EABH         PUBLIC        _GDispChipSel
  C:0DA4H         PUBLIC        _GDispSetPixel
  C:0ECBH         PUBLIC        GDispInit
  B:00A0H.4       PUBLIC        LCD_CS1
  B:00A0H.5       PUBLIC        LCD_CS2
  -------         PROC          GDISPINIT
  C:0ECBH         LINE#         86
  C:0ECBH         LINE#         87
  C:0ECBH         LINE#         88
  C:0ED0H         LINE#         89
  C:0ED3H         LINE#         90
  C:0ED8H         LINE#         91
  C:0EE0H         LINE#         92
  C:0EE5H         LINE#         93
  -------         ENDPROC       GDISPINIT
  -------         PROC          GDISPSWITCH
  B:0020H.0       SYMBOL        sw
  C:0EEAH         LINE#         110
  C:0EEAH         LINE#         111
  C:0EEAH         LINE#         112
  C:0EEFH         LINE#         113
  C:0F01H         LINE#         114
  -------         ENDPROC       GDISPSWITCH
  -------         PROC          _GDISPWRBYTE
  D:000CH         SYMBOL        col
  D:000DH         SYMBOL        page
  D:000EH         SYMBOL        c
  C:0E23H         LINE#         134
  C:0E29H         LINE#         135
  C:0E29H         LINE#         136
  C:0E2CH         LINE#         137
  C:0E2FH         LINE#         139
  C:0E36H         LINE#         140
  C:0E3DH         LINE#         142
  C:0E48H         LINE#         144
  C:0E5AH         LINE#         145
  C:0E62H         LINE#         146
  -------         ENDPROC       _GDISPWRBYTE
  -------         PROC          _GDISPCLR
  D:0009H         SYMBOL        pat
  -------         DO            
  D:000AH         SYMBOL        col
  D:000BH         SYMBOL        page
  -------         ENDDO         
  C:0E67H         LINE#         162
  C:0E69H         LINE#         163
  C:0E69H         LINE#         166
  C:0E6CH         LINE#         167
  C:0E6CH         LINE#         168
  C:0E81H         LINE#         169
  C:0E8AH         LINE#         170
  -------         ENDPROC       _GDISPCLR
  -------         PROC          _GDISPSETPIXEL
BL51 BANKED LINKER/LOCATER V5.03                                                      07/06/2006  17:26:57  PAGE 6


  D:0015H         SYMBOL        x
  D:0016H         SYMBOL        y
  B:0020H.1       SYMBOL        color
  -------         DO            
  D:0017H         SYMBOL        pre_data
  -------         ENDDO         
  C:0DA4H         LINE#         191
  C:0DA8H         LINE#         192
  C:0DA8H         LINE#         195
  C:0DABH         LINE#         196
  C:0DAEH         LINE#         198
  C:0DB5H         LINE#         199
  C:0DBCH         LINE#         201
  C:0DC7H         LINE#         203
  C:0DD7H         LINE#         204
  C:0DDAH         LINE#         205
  C:0DE1H         LINE#         206
  C:0DE8H         LINE#         207
  C:0DEBH         LINE#         209
  C:0E1EH         LINE#         211
  -------         ENDPROC       _GDISPSETPIXEL
  -------         PROC          _GDISPPIXSTRAT
  D:0009H         SYMBOL        x
  D:000AH         SYMBOL        y
  D:000BH         SYMBOL        pStr
  D:000EH         SYMBOL        fontSpace
  B:0020H.0       SYMBOL        color
  -------         DO            
  D:000FH         SYMBOL        pixelByte
  D:0010H         SYMBOL        bit_idx
  D:0011H         SYMBOL        i
  D:0012H         SYMBOL        c
  D:0013H         SYMBOL        fwidth
  D:0014H         SYMBOL        fheight
  -------         ENDDO         
  C:0C36H         LINE#         287
  C:0C40H         LINE#         288
  C:0C40H         LINE#         292
  C:0C4EH         LINE#         293
  C:0C4EH         LINE#         294
  C:0C5FH         LINE#         296
  C:0C71H         LINE#         297
  C:0C74H         LINE#         299
  C:0C85H         LINE#         300
  C:0C85H         LINE#         301
  C:0C88H         LINE#         302
  C:0C8EH         LINE#         303
  C:0C8EH         LINE#         305
  C:0CA1H         LINE#         306
  C:0CA1H         LINE#         307
  C:0CA4H         LINE#         308
  C:0CA4H         LINE#         310
  C:0CAEH         LINE#         311
  C:0CAEH         LINE#         312
  C:0CCDH         LINE#         313
  C:0CD7H         LINE#         314
  C:0CD7H         LINE#         315
BL51 BANKED LINKER/LOCATER V5.03                                                      07/06/2006  17:26:57  PAGE 7


  C:0CFFH         LINE#         316
  C:0D03H         LINE#         317
  C:0D07H         LINE#         319
  C:0D0FH         LINE#         320
  C:0D12H         LINE#         321
  -------         ENDPROC       _GDISPPIXSTRAT
  -------         PROC          GDISPRESET
  -------         DO            
  D:0007H         SYMBOL        i
  -------         ENDDO         
  C:0F63H         LINE#         335
  C:0F63H         LINE#         336
  C:0F63H         LINE#         339
  C:0F65H         LINE#         340
  C:0F6BH         LINE#         341
  C:0F6DH         LINE#         342
  C:0F73H         LINE#         343
  -------         ENDPROC       GDISPRESET
  -------         PROC          _GDISPCHIPSEL
  D:0007H         SYMBOL        wing
  C:0EABH         LINE#         359
  C:0EABH         LINE#         360
  C:0EABH         LINE#         361
  C:0EAEH         LINE#         362
  C:0EB3H         LINE#         363
  C:0EB6H         LINE#         364
  C:0EBBH         LINE#         365
  C:0EBEH         LINE#         366
  C:0EC3H         LINE#         367
  C:0EC6H         LINE#         368
  C:0ECAH         LINE#         369
  -------         ENDPROC       _GDISPCHIPSEL
  C:0F0AH         SYMBOL        L?0066
  -------         PROC          L?0065
  -------         ENDPROC       L?0065
  C:0F0AH         SYMBOL        L?0066
  -------         PROC          GDISPWR
  B:0020H.2       SYMBOL        type
  D:0018H         SYMBOL        dat
  C:0F0EH         LINE#         384
  C:0F0EH         LINE#         385
  C:0F0EH         LINE#         386
  C:0F17H         LINE#         387
  C:0F19H         LINE#         388
  C:0F1BH         LINE#         389
  C:0F1EH         LINE#         390
  C:0F1FH         LINE#         391
  C:0F21H         LINE#         392
  -------         ENDPROC       GDISPWR
  -------         PROC          GDISPRD
  B:0020H.2       SYMBOL        type
  -------         DO            
  D:0007H         SYMBOL        lcd_status
  -------         ENDDO         
  C:0F3BH         LINE#         407
  C:0F3BH         LINE#         408
  C:0F3BH         LINE#         411
BL51 BANKED LINKER/LOCATER V5.03                                                      07/06/2006  17:26:57  PAGE 8


  C:0F3EH         LINE#         412
  C:0F47H         LINE#         413
  C:0F49H         LINE#         414
  C:0F4BH         LINE#         415
  C:0F4CH         LINE#         416
  C:0F4EH         LINE#         417
  C:0F50H         LINE#         419
  C:0F50H         LINE#         420
  -------         ENDPROC       GDISPRD
  -------         PROC          GDISPBACKLITE
  B:0020H.0       SYMBOL        ctrl
  C:0F80H         LINE#         434
  C:0F80H         LINE#         435
  C:0F80H         LINE#         436
  C:0F88H         LINE#         437
  -------         ENDPROC       GDISPBACKLITE
  -------         ENDMOD        KS0108

  -------         MODULE        ?C?CLDPTR
  C:0F22H         PUBLIC        ?C?CLDPTR
  -------         ENDMOD        ?C?CLDPTR

*** WARNING L16: UNCALLED SEGMENT, IGNORED FOR OVERLAY PROCESS
    SEGMENT: ?PR?_DELAYUS?DELAY

******************************************************************************
* RESTRICTED VERSION WITH 0800H BYTE CODE SIZE LIMIT; USED: 078FH BYTE (94%) *
******************************************************************************

Program Size: data=26.3 xdata=0 code=1932
LINK/LOCATE RUN COMPLETE.  1 WARNING(S),  0 ERROR(S)
